:100000000C940E060C942B060C942B060C942B06C9
:100010000C942B060C942B060C942B060C942B069C
:100020000C942B060C942B060C9466270C94382801
:100030000C94AF210C942B060C942B060C942B06DD
:100040000C942B060C942B060C942B060C942B066C
:100050000C942B060C9437220C942B060C942B0634
:100060000C942B060C942B060C942B060C942B064C
:100070000C942B060C942B060C942B060C942B063C
:100080000C942B060C942B060C942B060C942B062C
:100090000C942B060C942B060C942B060C942B061C
:1000A0000C942B060C942B060C942B06F909F909D9
:1000B000250A250A8D0AAB0AC30BC30BB60A4F0BE0
:1000C000600B600BA528CC28C429CC28C42918298A
:1000D0003B29C4299229A1290152540055005600F8
:1000E000010000000000000000000000000000000F
:1000F0000000000000005F00600061005700010088
:1001000000000000000000000000000000000000EF
:10011000000000005C005D005E0057000100000070
:1001200000000000000000000000000000000000CF
:10013000000059005A005B00580001000000000058
:1001400000000000000000000000000000000000AF
:10015000620062006300580001000000000000001F
:10016000000000000000000000000000000001008E
:100170001E001F0020002100220023002400250073
:1001800026002700010001000100010029001400E1
:100190001A000800150017001C0018000C001200BF
:1001A00013002A005F00600061002B0004001600AD
:1001B000070009000A000B000D000E000F003300BD
:1001C00034005C005D005E00E1001D001B000600C5
:1001D00019000500110010003600370038002862B1
:1001E00059005A005B00E000E300E200E200025127
:1001F000E1002C000351E700E6004C00E40062003F
:100200006200630001000100010001000100010023
:1002100001000100010001000100010001000100D6
:10022000010001003A003B003C003D003E003F0061
:100230004000410042004300530054005500560066
:1002400035001E001F002000210022002300240092
:1002500025002600270001000100010057000100D1
:10026000440045000100010001002800E500E7000E
:1002700037642A61010001000100580001000100FB
:1002800001000100010001002800E500010001005B
:100290000100010001000100010001000100010056
:1002A0000100010001000100010001000100010046
:1002B0000100010001000100005C2B005200010060
:1002C0004900E000E1004B004A002D002E004C00E8
:1002D0000100010001003900500051004F004600AC
:1002E000E100E0004E004D002F0030003100010021
:1002F00001000100010048000100010001000100AF
:1003000001000100E700E60001000100010001001A
:100310000100005201000100010001000100010084
:1003200001000100010001000100010001000100C5
:1003300044454255473A2064697361626C65642E96
:100340000A0044454255473A20656E61626C656417
:100350002E0A000A0025303258006C65645F746113
:10036000736B3A20004F6E6573686F743A20616357
:10037000746976653A2025640A000A002530313612
:1003800062003A200025303258000A722F63203074
:100390003132333435363738394142434445460AE1
:1003A00000290A002575002F002575005D2800250D
:1003B00064002000256400200025640020002564DE
:1003C000007C0025303258006D6F7573656B657960
:1003D000205B62746E7C782079207620685D2872BC
:1003E00065702F61636C293A205B00313A096465BE
:1003F0006C6179282A31306D73293A2025750A32CB
:100400003A09696E74657276616C286D73293A20B9
:1004100025750A333A096D61785F73706565643AD2
:100420002025750A343A0974696D655F746F5F6DD4
:1004300061783A2025750A353A09776865656C5FF9
:100440006D61785F73706565643A2025750A363A88
:1004500009776865656C5F74696D655F746F5F6D62
:1004600061783A2025750A00703A097072696E74D5
:100470002076616C7565730A643A0973657420644B
:10048000656661756C74730A75703A092B310A647C
:100490006E3A092D310A6C743A092B31300A7274A4
:1004A0003A092D31300A4553432F713A0971756964
:1004B000740A0A7370656564203D2064656C74611C
:1004C000202A206D61785F7370656564202A20287A
:1004D000726570656174202F2074696D655F746F3B
:1004E0005F6D6178290A77686572652064656C7450
:1004F000613A20637572736F723D25642C207768B2
:1005000065656C3D25640A53656520687474703AAE
:100510002F2F656E2E77696B6970656469612E6F28
:1005200072672F77696B692F4D6F7573655F6B65A8
:1005300079730A004D3E20004D25753A25733E2003
:10054000003F0A003D2025750A003F0A00646566E9
:1005500061756C74730A0025750A003F0A000A0968
:100560002D2056616C756573202D0A00710A000AF2
:10057000092D204D6F7573656B6579202D0A003F3D
:1005800000433E20004C25640A000A092D205374C4
:1005900061747573202D0A686F73745F6B6579627F
:1005A0006F6172645F6C65647328293A202530326C
:1005B000580A6B6579626F6172645F70726F746FF5
:1005C000636F6C3A20253032580A6B6579626F612F
:1005D00072645F69646C653A20253032580A746928
:1005E0006D65725F72656164333228293A20253067
:1005F000386C580A000A092D2056657273696F6EAF
:10060000202D0A5649443A20307834303235286457
:100610006930696229205049443A203078303542A7
:10062000352854686520357835204B6579626F61CF
:10063000726429205645523A203078303130300AE1
:100640004255494C443A20202846656220323720E2
:1006500032303232290A4F5054494F4E533A204CCF
:10066000554641204D4F5553454B4559204558540B
:1006700052414B455920434F4E534F4C4520434F19
:100680004D4D414E4420343039360A4743433A20D9
:10069000352E342E30204156522D4C4942433A20BB
:1006A000322E302E30204156525F415243483A207C
:1006B000617672350A000A092D20436F6E736F6CE4
:1006C00065202D0A4553432F713A09717569740AE3
:1006D0006D3A096D6F7573656B65790A000A092DAE
:1006E000204D61676963202D0A443A0944656275AB
:1006F00067204D65737361676520546F67676C652C
:100700000A583A094D6174726978204465627567C8
:10071000204D6F646520546F67676C65202D2053F2
:10072000686F77206B657970726573736573206984
:100730006E206D617472697820677269640A4B3A41
:10074000094B6579626F6172642044656275672048
:10075000546F67676C65202D2053686F77206B6539
:10076000797072657373207265706F72740A4D3A96
:10077000094465627567204D6F75736520546F6716
:10078000676C650A563A0956657273696F6E0A534B
:100790003A095374617475730A433A094163746981
:1007A0007661746520436F6E736F6C65204D6F6466
:1007B000650A46312D4631303A09537769746368CA
:1007C00020746F204C6179657220302D39202846C5
:1007D0003130203D204C30290A302D393A095377E9
:1007E0006974636820746F204C6179657220302DC4
:1007F000390A47524156453A09537769746368206C
:10080000746F204C6179657220302028616C7465AA
:10081000726E617465290A423A094A756D702074D6
:100820006F20426F6F746C6F616465720A45534349
:100830003A094A756D7020746F20426F6F746C6F47
:10084000616465722028616C7465726E61746529DB
:100850000A453A095072696E7420454550524F4D11
:100860002053657474696E67730A4253504143455F
:100870003A09436C65617220454550524F4D0A005C
:100880006B65796D61705F636F6E6669672E72610B
:10089000773A20253032580A2E737761705F636F84
:1008A0006E74726F6C5F636170736C6F636B3A2010
:1008B00025750A2E636170736C6F636B5F746F5F75
:1008C000636F6E74726F6C3A2025750A2E737761B0
:1008D000705F6C63746C5F6C6775693A2025750A8C
:1008E0002E737761705F7263746C5F726775693ABB
:1008F0002025750A2E737761705F6C616C745F6C74
:100900006775693A2025750A2E737761705F726189
:100910006C745F726775693A2025750A2E6E6F5F79
:100920006775693A2025750A2E737761705F677263
:100930006176655F6573633A2025750A2E7377616A
:10094000705F6261636B736C6173685F6261636B3C
:1009500073706163653A2025750A2E6E6B726F3A6B
:100960002025750A0064656275675F636F6E66694E
:10097000672E7261773A20253032580A2E656E61F3
:10098000626C653A2025750A2E6D61747269783A39
:100990002025750A2E6B6579626F6172643A202595
:1009A000750A2E6D6F7573653A2025750A006565A9
:1009B000636F6E6669673A0A64656661756C745F39
:1009C0006C617965723A2025750A003F000A6D6FE7
:1009D0007573653A206F66660A000A6D6F757365F8
:1009E0003A206F6E0A000A6B6579626F6172643A31
:1009F000206F66660A000A6B6579626F6172643AFD
:100A0000206F6E0A000A6D61747269783A206F6611
:100A1000660A000A6D61747269783A206F6E0A0086
:100A20000A64656275673A206F66660A000A646543
:100A30006275673A206F6E0A000A0A4A756D70691E
:100A40006E6720746F20626F6F746C6F6164657283
:100A50002E2E2E2000433E2000436C656172696E8D
:100A60006720454550524F4D0A000A002530325844
:100A700020006B6579626F6172645F7265706F727E
:100A8000743A20005B735D005B575D005B535D0053
:100A90005B525D005B445D005B435D0022035400DC
:100AA00068006500200035007800350020004B000C
:100AB0006500790062006F00610072006400000050
:100AC0000C03640069003000690062000000040348
:100AD000090409025B00030100A0FA0904000001F7
:100AE00003010100092111010001224000070581D5
:100AF000030800010904010001030000000921119D
:100B0000010001227B000705820320000109040285
:100B10000002030000000921110100012222000748
:100B200005830320000107050303200001120100D3
:100B300002000000082540B5050001010200010681
:100B400031FF0974A1010975150026FF0095207574
:100B50000881020976150026FF009520750891028C
:100B6000C005010902A10185020901A100050919B9
:100B70000129081500250195087501810205010963
:100B80003009311581257F950275088106093815D0
:100B900081257F950175088106050C0A38021581AB
:100BA000257F950175088106C0C005010980A10156
:100BB000850319012AB700150126B70095017510A4
:100BC0008100C0050C0901A101850419012AA002B8
:100BD000150126A002950175108100C005010906C6
:100BE000A101050719E029E7150025019508750100
:100BF00081029501750881010507190029FF15007B
:100C000026FF00950675088100050819012905953C
:100C10000575019102950175039101C011241FBE54
:100C2000CFEFDAE0DEBFCDBF11E0A0E0B1E0E4E05D
:100C3000F5E502C005900D92AC3FB107D9F722E06F
:100C4000ACEFB1E001C01D92A23FB207E1F70E94F4
:100C500006180C94802A0C940000FF93EF93E09107
:100C6000FC01F091FD01309709F00995EF91FF919A
:100C70000895FC018591803011F0EFDFFBCF0895DE
:100C8000FF27E0E230E247FF0CC0419597FF09C023
:100C9000EDE26095709580959095611D711D811DA7
:100CA000911D27FF02C0219530E350E2AA27660F6D
:100CB000771F881F991FAA1FA41710F0A41B639504
:100CC0005A95A9F7AA3008F0A95FA05DAF93F395F4
:100CD000611571058105910541F7ED3211F4EF932E
:100CE000F395F21718F43F93F395FBCF8F91B5DF8F
:100CF000FA95E1F70895E991F9918591803021F015
:100D0000853219F0AADFF9CF089520E0E8945591D3
:100D10005532C1F3503311F4689455915A3348F465
:100D2000505390F3220F022E220F220F200D250F79
:100D3000F4CF0EF4219589919991533619F35337D5
:100D400029F1533559F1BC0188279927E8945C367D
:100D500021F48991999168945591543639F446EF6C
:100D60007EF077FF0DC08FEF9FEF0AC055374AE046
:100D700039F0583540E121F0523642E009F008954B
:100D8000FF93EF937DDFEF91FF91B7CFFF93EF9349
:100D9000FC0181918030B9F360DFFBCFFF93EF93CB
:100DA00068DFF1CFDF93CF93CDB7DEB72596A3DF12
:100DB000CF91DF91089581E0089581E008950C942A
:100DC000DD0608950C94E1061F93CF93DF9300D0C6
:100DD00000D01F92CDB7DEB749835A836B83309121
:100DE000FF0189819A81311114C0662359F02223B1
:100DF00049F00E94000E182F682F89819A810E9465
:100E0000A90D03C00E94D40D182F69817A81812F0A
:100E100004C00E94000E69817A810F900F900F909C
:100E20000F900F90DF91CF911F910C944415FC010E
:100E3000262F408151816281738184810C94E40664
:100E400081E00895CF93DF93EC0160E00E941707E3
:100E5000BE01DF91CF910C94E2060C94B7160C946E
:100E6000B31608950E94530C0E9431072FEF84E3BC
:100E70009CE0215080409040E1F700C000000C94BD
:100E80005D220F931F93CF93DF938C0161E00E944B
:100E90001707EC01B8010E94DF06882309F45BC044
:100EA000B801CE010E943C20882309F454C0B80147
:100EB000CE010E941E1B882309F44DC0B801CE014B
:100EC0000E94981F882309F446C0F8018281882374
:100ED000D9F1CF3D8CE5D80779F140F4C115FCE597
:100EE000DF0791F0C130DC4591F02EC0CC35EDE547
:100EF000DE0741F1CD35FDE5DF0709F1CB35DD45F5
:100F000019F50E94971220C00E94320724C08091D8
:100F10009802C82FC095C170C0FB80F980939802D9
:100F2000CC2329F082E493E00E94390614C080E3C8
:100F300093E00E94390610C00E9445130CC00E9425
:100F40008E1202C00E949A12C801DF91CF911F91A8
:100F50000F910C94DB06C0E08C2FDF91CF911F9195
:100F60000F9108950E9491210C94F0070E94F307BD
:100F70000C9497218295982F937344E0949F90014D
:100F800011248C7C86958695282B822F8575880F59
:100F90002A7A2695822B0895CF93DF93D92F0E942A
:100FA000BA07C82F8D2F0E94BA072C2F30E0322F9E
:100FB0002227A901482BCA01DF91CF9108950895F6
:100FC0000C94DF0781E008950C94E2070895CF9315
:100FD000C82F0E94E0078C2F0E94E407CF9108954C
:100FE00080E00C94E7070E9498200C94E707CF93C9
:100FF0000E949820C82F8091FE01C81741F1C0932C
:10100000FE018091980282FF1EC080FF04C08AE525
:1010100093E00E9439068091980280FF0CC01F92D5
:10102000CF9385E593E09F938F930E94D2060F9014
:101030000F900F900F908091980280FF04C083E57D
:1010400093E00E9439068C2FCF910C94E707CF9143
:101050000895CF93DF93CDB7DEB72B970FB6F894F3
:10106000DEBF0FBECDBF4F83588769877A878B87D6
:1010700061110E94C6119E012F5F3F4F86E0F9016A
:1010800011928A95E9F785E0FE013796D901019022
:101090000D928A95E1F789819A814C815D81452B7A
:1010A00031F09F3F31F491E08F3F19F403C091E09C
:1010B00001C090E090FF09C049815A816B817C8119
:1010C0008D819E810E94E71005C0C9010E94200702
:1010D0008111F2CF2B960FB6F894DEBF0FBECDBFB5
:1010E000DF91CF910895FC01808191810E94420E91
:1010F0000895CF93882309F4A9C0C82F8238C1F47A
:101100000E94982081FDA2C069E380910201909124
:1011100003010E9469210E94E8112FEF81EE94E003
:10112000215080409040E1F700C0000069E319C001
:10113000833801F50E94982080FD88C063E5809186
:101140000201909103010E9469210E94E8112FEF92
:1011500081EE94E0215080409040E1F700C0000013
:1011600063E580910201909103010E946B21CF9170
:101170000C94E8118438C1F40E94982082FD66C066
:1011800067E480910201909103010E9469210E940D
:10119000E8112FEF81EE94E0215080409040E1F77C
:1011A00000C0000067E4DDCF8CEF8C0F813AF8F4CB
:1011B0008C2F0E94411F811149C06C2F8091020128
:1011C000909103010E943321882349F06C2F809174
:1011D0000201909103010E946B210E94E8116C2F83
:1011E00080910201909103010E946921C0CF80E2A9
:1011F0008C0F883048F4C77081E001C0880FCA9511
:10120000EAF70E94A911B3CFEBE5EC0FE33040F40D
:10121000F0E0E95BFE4F808190E0CF910C94FB20E1
:10122000E8E5EC0FE73150F4F0E0EE0FFF1FE75E6A
:10123000FE4F80819181CF910C941121CD3E30F0F1
:101240008C2F0E948B18CF910C945D19CF9108952B
:10125000882309F464C0823879F40E94982081FFC1
:101260005EC069E380910201909103010E946921AF
:101270000E94E81169E310C08338B1F40E949820FD
:1012800080FF4DC063E580910201909103010E94AF
:1012900069210E94E81163E58091020190910301A8
:1012A0000E946B210C94E811843879F40E949820F4
:1012B00082FF35C067E480910201909103010E9492
:1012C00069210E94E81167E4E7CF9CEF980F913AFB
:1012D00010F4682FE1CF90E2980F983050F48770A7
:1012E00091E001C0990F8A95EAF7892F0E94AF110A
:1012F000D9CF9BE5980F933020F480E090E00C94D8
:10130000FB2098E5980F973120F480E090E00C9452
:1013100011218D3E20F00E94E6180C945D1908956D
:101320001F93CF93DF93182FEB010E94790820972A
:1013300041F08FE99FE00197F1F700C0000021978D
:10134000F6CF812FDF91CF911F910C94280989331B
:1013500019F060E070E002C060E570E00C94900964
:10136000882321F00E94A9110C94E8110895882384
:1013700021F00E94AF110C94E8110895CF92DF92F2
:10138000EF92FF920F931F93CF93DF937C01D62FA1
:10139000C72FFC011281058102950F700E949F11D9
:1013A0008823B9F01123A9F08C2F807F803421F09D
:1013B00080E28D0F883068F08091CC0282FD09C0F8
:1013C00082E00E9448120E949F1191E0D82ED926F7
:1013D00001C0D12CCC2EC2948FE0C8228C2D90E07D
:1013E0008C30910508F0CFC1FC01EA5AFF4F0C94F4
:1013F000172A8C2F807FCF70882311F0C295C07F71
:10140000112399F0CC2309F4AAC180E28D0F883012
:1014100010F0D11104C08C2F0E94A91103C08C2F91
:101420000E94B9110E94E8119AC18D2F0E942809CB
:10143000CC2309F4A8C180E28D0F883038F1DD2378
:1014400029F18C2F0E94BF1124C08C2F807FCF7078
:10145000803211F0C295C07FDD2319F0D130A1F1A7
:101460003DC08091CC0282FF17C0112349F0CC23EC
:1014700029F08C2F0E94A9110E94E81180E070C110
:1014800080E00E942809CC2309F47DC18C2F0E94A2
:10149000AF110E94E81177C1112371F0002341F0D0
:1014A000013031F40E94C9118C2B0E94D1116BC103
:1014B0000E94C9118C2B1DC0002319F0013009F4C2
:1014C00062C10E94DE1125C0112321F0063008F010
:1014D0005AC10EC0053008F056C11BC0112361F07F
:1014E000002331F0F701858180FF39C18F7085833A
:1014F0008C2F0E94B00947C1002359F0D93309F05D
:101500003FC1FFEF07EE13E0F15000401040E1F75C
:1015100035C18C2F0E94B70936C18C2F86958695D0
:10152000837019F0813061F02EC1112321F08D2FCD
:101530009C2F937002C080E090E00E94FB202BC1A2
:10154000112321F08D2F9C2F937002C080E090E03A
:101550000E94112120C18D2F112319F00E948B1898
:1015600002C00E94E6180E945D1915C18C2F83707D
:1015700009F047C011110BC12D2F22952695277018
:10158000220F220F6D2F6F70862F90E0A0E0B0E049
:10159000022E04C0880F991FAA1FBB1F0A94D2F7FE
:1015A000D4FF10C04FE050E060E070E004C0440F92
:1015B000551F661F771F2A95D2F740955095609565
:1015C000709503C040E050E0BA01C695C695C3705F
:1015D0008A019B01082B192B2A2B3B2BC901B8012F
:1015E000C23049F058F4C13019F00E94BF0CCFC08E
:1015F0000E94AD0CCCC00E94D10CC9C00E94AB0CA3
:10160000C6C0112319F08C2F817001C086958823E4
:1016100009F4BDC02D2F229526952770220F220F89
:101620006D2F6F70862F90E0A0E0B0E0022E04C016
:10163000880F991FAA1FBB1F0A94D2F7D4FF10C0AE
:101640004FE050E060E070E004C0440F551F661F9B
:10165000771F2A95D2F7409550956095709503C0F5
:1016600040E050E0BA01C695C695C3708A019B015F
:10167000082B192B2A2B3B2BC901B801C23049F08A
:1016800058F4C13019F00E94840D81C00E94720D7F
:101690007EC00E94960D7BC00E94E50C78C0CF7082
:1016A000112339F08C2F0E940B0D8D2F0E94B00951
:1016B0006EC08D2F0E94B7098C2F0E942C0D67C021
:1016C000D23F21F128F4D03F41F0D13FC1F043C0D7
:1016D000D33F19F1D43F79F03EC0112341F00530DA
:1016E00008F051C08C2F8F710E94510D4CC00630F4
:1016F00008F049C0F7CF8091CC0282FF18C01123B7
:1017000039F08C2F8F710E940B0D3DC01123C9F34E
:101710008C2F8F710E942C0D36C0112329F08C2F35
:101720008F710E94F60C2FC00E94F10C2CC0112367
:1017300049F0CF718C2F0E940B0D63E08C2F0E941B
:101740002D1221C081E00E9448120230E0F082E0B8
:101750000E94481218C0112331F0002391F28D2FFE
:101760000E94790810C0002399F2D93349F41FEF81
:1017700027EE33E0115020403040E1F700C0000078
:101780008D2F0E94280988EF8C0D843020F40E9450
:1017900098200E94E707DD20C9F00E949B1180FD80
:1017A00015C0F70112820E9495110E940B0DC7010E
:1017B0000E94070C0E949511DF91CF911F910F910C
:1017C000FF90EF90DF90CF900C942C0DDF91CF9194
:1017D0001F910F91FF90EF90DF90CF9008950F939E
:1017E0001F93CF93DF93EC01688179818A810E94F6
:1017F0004D0E8C010E94A80D0E94990CB801CE01DB
:101800000E94BE09DF91CF911F910F910895CF9350
:10181000DF93EC01988189812B813C81232B31F06E
:101820008F3F31F481E09F3F19F403C081E001C094
:1018300080E080FD1DC0CE010E944107811110C0D3
:101840000E949F118823A1F08A81882389F08091CA
:10185000CC0282FD0DC082E0DF91CF910C94481242
:10186000CE010E94EF0BCE01DF91CF910C942207A5
:10187000DF91CF91089580E090E00E94FB2080E00E
:1018800090E00E9411210E94C6110E94E8110E945E
:10189000101B0C945D1980910201909103010E942C
:1018A0006D210C943B0C0E94B6110C944B0C92953C
:1018B0009F70963079F010F4925001C09A50923097
:1018C00068F4803F69F018F4883E40F409C0843F12
:1018D00029F406C0883E20F0813F11F080E0089591
:1018E00081E00895FC01808191810E94420E0E9456
:1018F000570C0895CF93DF9300D000D01F92CDB73F
:10190000DEB70F900F900F900F900F90DF91CF9157
:101910000895CF93DF9300D000D000D0CDB7DEB7CD
:1019200026960FB6F894DEBF0FBECDBFDF91CF91E4
:101930000895089508950C949A0C0C949B0C0E94A1
:101940009D0C609336027093370280933802909317
:1019500039020C943B0C0C949F0C0F931F93009135
:101960003602109137022091380230913902602BF3
:10197000712B822B932B1F910F910C949F0C0F9323
:101980001F93009136021091370220913802309156
:10199000390260237123822393231F910F910C94AA
:1019A0009F0C0F931F9300913602109137022091E4
:1019B00038023091390260277127822793271F91BF
:1019C0000F910C949F0C0C949A0C0E94E30C609362
:1019D00032027093330280933402909335020C9458
:1019E0003B0C60E070E0CB010C94E50C0F931F936F
:1019F00041E050E060E070E08A019B0104C0000F0C
:101A0000111F221F331F8A95D2F7C901B8011F91F8
:101A10000F910C94E50C0F931F9341E050E060E0B0
:101A200070E004C0440F551F661F771F8A95D2F7D8
:101A30008091320290913302A0913402B09135022C
:101A40008A019B01082B192B2A2B3B2BC901B801BA
:101A50001F910F910C94E50C0F931F9341E050E000
:101A600060E070E004C0440F551F661F771F8A9521
:101A7000D2F7409550956095709580913202909183
:101A80003302A0913402B09135028A019B010823F0
:101A900019232A233B23C901B8011F910F910C94EC
:101AA000E50C0F931F9341E050E060E070E004C04C
:101AB000440F551F661F771F8A95D2F78091320217
:101AC00090913302A0913402B09135028A019B01BA
:101AD000082719272A273B27C901B8011F910F9111
:101AE0000C94E50C0F931F93009132021091330276
:101AF0002091340230913502602B712B822B932B75
:101B00001F910F910C94E50C0F931F9300913202DB
:101B100010913302209134023091350260237123F9
:101B2000822393231F910F910C94E50C0F931F9325
:101B3000009132021091330220913402309135022B
:101B400060277127822793271F910F910C94E50C32
:101B500008952FE0929F800D1124E82FE695E695D9
:101B6000E695877051E001C0550F8A95EAF785E048
:101B7000E89FF0011124E050FE4F20E030E070E0DB
:101B80004081CB01022E02C0969587950A94E2F718
:101B90008170819584278523842781932F5F3F4F10
:101BA0002530310569F708952FE0929F800D1124AB
:101BB000682F669566956695982F977085E0689F63
:101BC000B001112440E050E080E0FB01E40FF51F7C
:101BD000E050FE4F208130E0092E02C03695279557
:101BE0000A94E2F721703327042E01C0220F0A94D1
:101BF000EAF7822B4F5F5F4F4530510531F708956B
:101C0000BF92CF92DF92EF92FF920F931F93CF93E9
:101C1000DF938C01C0903202D0903302E090340206
:101C2000F09035028091360290913702A0913802EF
:101C3000B0913902C82AD92AEA2AFB2ACFE1D0E09A
:101C4000D701C6010C2E04C0B695A7959795879528
:101C50000A94D2F780FD04C0219790F7B12C07C0F9
:101C6000BC2EB8018C2F0E9457150197A9F38B2D1C
:101C7000DF91CF911F910F91FF90EF90DF90CF9068
:101C8000BF900895CF93DF93EC010E94000EBE0138
:101C90000E945715DF91CF9108951F93CF93DF9343
:101CA000EB019091FF01992321F0CB010E94420E9C
:101CB00013C0882349F0CB010E94000E182F682F13
:101CC000CE010E94A90D04C0CB010E94D40D182F93
:101CD000BE01812F0E945715DF91CF911F9108956A
:101CE0001F93CF93DF93C0913A0216E080913B029D
:101CF000C81799F0D0E01C9FF0011D9FF00D112432
:101D0000E45CFD4F408151816281738184819581C2
:101D10000E94890C2196C770E9CFDF91CF911F9166
:101D2000089540916C0250916D0260916E02709125
:101D30006F0280917002909171020C94890CEF9265
:101D4000FF920F931F93CF93DF938091710282953F
:101D50008F7009F065C080916E02882309F460C01D
:101D600080913A02F0903B0210916C0200916D025A
:101D700060916F027091700291E01F3F09F090E056
:101D8000C0910001D0910101292F96E0E92E8F1515
:101D900009F446C06115710521F00F3F21F030E0D4
:101DA00003C031E001C0322F90E030FD36C0E89E24
:101DB000F001E99EF00D1124DF01A45CBD4F1196E6
:101DC0003C911197301329C03C91311326C01296D3
:101DD0003C911297311121C013964D915C9114974B
:101DE000461B570B4C175D07C0F4809171028F7032
:101DF000806180937102EF5BFD4F80818F70806105
:101E000080838CE692E00E94070CDF91CF911F91B6
:101E10000F91FF90EF900C94700E01968770B7CFE2
:101E2000DF91CF911F910F91FF90EF9008959F92B6
:101E3000AF92BF92CF92DF92EF92FF920F931F93D8
:101E4000CF93DF93CDB7DEB761970FB6F894DEBFBF
:101E50000FBECDBF8C0185E0F801DE011D9601901B
:101E60000D928A95E1F7D8011296EC9090916C0250
:101E7000E0916D0220916F023091700221153105C1
:101E800031F0EF3F31F481E09F3F19F403C081E06E
:101E900001C080E0B82FB1709B2E80FD47C1D801F2
:101EA0004C9111965C9111971396AD90BC9014973C
:101EB0008CE6C82E82E0D82EF0906E02B501621B2F
:101EC000730B2091000130910101FF2009F4D9C06A
:101ED000809171026217730708F095C0282F207F48
:101EE00009F052C05E1313C0491311C0FE2CE1105B
:101EF0000EC08F708061809371020E94910EC601A6
:101F00000E94070C80917102F80185834DC1AB28B6
:101F100031F05F3F31F481E04F3F19F403C081E0BD
:101F200001C080E080FD03C081E08E2502C080E01A
:101F300090E0F82FF170FF2E80FF1CC080913A02D4
:101F400020913B0236E0821709F40BC190E0389FE4
:101F5000F001399FF00D1124E45CFD4F61815613AF
:101F600006C06081461303C06281E61203C0019679
:101F70008770E9CFFE2CEE2009F416C18091710222
:101F800081608093710254C05E1306C0491304C07F
:101F9000E11002C0F80199C0C8010E94720C8823A8
:101FA00061F1EE2051F120917102822F82958F70A4
:101FB00090E0029774F080916C0290916D02988786
:101FC0008F831986BB86AA862C87CE0107960E942E
:101FD000070C86E0F801ACE6B2E001900D928A951C
:101FE000E1F70E949F0E0E94910E0AC05E1711F148
:101FF000C8010E94720C81112CC0C8010E94070CFC
:10200000FF24F394D1C0282F207F81F77A2DB98A3D
:10201000A88A6E2D89890E947A0C8CE692E00E9433
:10202000070C86E0D6011D928A95E9F70E94910E71
:10203000F12CBAC04913DCCFE110DACFF801858367
:10204000C8010E94070C86E0D6011D928A95E9F727
:10205000ABC0EE2091F220917102822F82958F7099
:1020600090E002970CF4B5CF80916C0290916D02D4
:102070009A8389831B82BD82AC822E83CE01019616
:10208000A6CF6217730708F044C0FE2CEE2009F4B7
:10209000B4CF5E1330C049132EC02091710220FDD1
:1020A00021C0822F82958F70482F50E04115510535
:1020B000C9F0F80125834F30510541F08F5F982F0B
:1020C0009295907F822F8F70892B8583C8010E9403
:1020D000070C86E0F801ACE6B2E001900D928A951B
:1020E000E1F73CC086E0F801ACE6B2E001900D9269
:1020F0008A95E1F759C0C8010E94720C811169CF1D
:1021000080917102816080937102C8010E94070C66
:102110004BC07A2DB98AA88A6E2D89890E947A0CC3
:1021200086E0D6011D928A95E9F718C0EE2009F4E1
:1021300064CFC8010E94720CF82E882309F45DCF89
:1021400086E0F801ACE6B2E001900D928A95E1F7E5
:102150008CE692E00E9473080E949F0E0E94910EEE
:1021600023C04D875E878D859E850E94420E292F54
:1021700022952F70223028F49F7039F0811105C00C
:102180000BC0243028F49F7049F4805E883020F022
:10219000C8010E94070C9F2CF92C06C0D801159687
:1021A0009C91907F91F7F8CF8F2D61960FB6F894A0
:1021B000DEBF0FBECDBFDF91CF911F910F91FF907A
:1021C000EF90DF90CF90BF90AF909F9008951F93B6
:1021D000CF93DF93CDB7DEB72C970FB6F894DEBF61
:1021E0000FBECDBF4F83588769877A878B879C87BF
:1021F000CE0107960E94170F8823D1F09F81888512
:102200002A853B85232B31F08F3F31F481E09F3FBE
:1022100019F403C081E001C080E080FD47C04F8118
:10222000588569857A858B859C850E94890C3EC07E
:1022300086E0FE013796DE01119601900D928A9597
:10224000E1F7FF81E8856A857B856115710531F0CD
:10225000EF3F31F481E0FF3F19F403C081E001C09A
:1022600080E080FD23C020913B0230E0C90101964F
:102270008770992740913A0250E084179507F1F151
:10228000F983EA837D836C8396E0929FD001939FCC
:10229000B00D1124A45CBD4FFE01319601900D924A
:1022A0009A95E1F780933B020E94700E16E08091B0
:1022B0003A0290913B02891771F1189FC0011124D5
:1022C000845C9D4F0E94170F882329F1E0913A0208
:1022D0001E9FF0011124E45CFD4F40815181628119
:1022E0007381848195810E94890C80913A0290E0EB
:1022F00001968770992780933A02D9CF0E94530C98
:1023000010923B0210923A02ECE6F2E086E0DF0126
:102310001D928A95E9F72C960FB6F894DEBF0FBE92
:10232000CDBFDF91CF911F91089580917A0285955D
:1023300085958595089580917A028770089590918A
:102340007A02977081E009F480E008958091850217
:10235000089590918502892B809385020895809538
:1023600090918502892380938502089510928502B9
:10237000089590918402892B80938402089580951A
:10238000909184028923809384020895109284029C
:10239000089580917B02089508950C94CC110C94BB
:1023A000CD119091CC0292FD08C090917B029817BC
:1023B00021F080937B020C94CF11089580917B02D1
:1023C000882329F010927B0280E00C94CF110895AD
:1023D000CF93DF93E0910201F09103018091850298
:1023E0008083E0910201F091030190818091840249
:1023F000892B808380917B02882381F0E091020108
:10240000F09103019081892B80838091020190914A
:1024100003010E94272181110E94DE11C091020157
:10242000D091030148E050E062E772E0CE010E94E3
:10243000312A892B69F088E0FE01A2E7B2E0019021
:102440000D928A95E1F7CE01DF91CF910C94A420F3
:10245000DF91CF9108950C94CC119091CC0292FD14
:1024600010C098E0899F90011124262B20937A02B6
:102470000E940B0D80917A028595859585950C9427
:102480002B120C940B0D10927A0280E00C942B12FC
:1024900020917A028095822380937A02982F9770F8
:1024A00099F430E0482F082E000C550B24173507FF
:1024B00059F09091CC0292FD07C085958595859540
:1024C0000E942C0D0C9443120895CF939091CC024E
:1024D00092FB222720F92817F9F0C82F892FC0FB7B
:1024E00082F98093CC028091CB029091CC020E9421
:1024F000C11282E00E9448128091980280FF0CC0B5
:102500001F92CF9385E693E09F938F930E94D2060C
:102510000F900F900F900F90CF9108958091CC0263
:1025200082FB882780F991E089270C94651281E06D
:102530000C94651280E00C94651280E090E00E949B
:10254000462A21E0893E9E4F09F020E0822F08951F
:1025500082E090E00C943E2A83E090E00C943E2AC6
:10256000CF9384E090E00E943E2AC82F82E290E060
:102570000E943E2A2C2F30E0A901582BCA01CF918E
:102580000895CF93C92F682F84E090E00E944C2AD1
:102590006C2F82E290E0CF910C944C2AAB01BC01ED
:1025A0008FE090E00C945E2AAB01BC0183E190E0E7
:1025B0000C945E2A60E070E0CB010C94D41260E0D1
:1025C00070E0CB010E94CE120C94DA1269EE7EEF1D
:1025D00080E090E00E946A2A60E082E090E00E9441
:1025E0004C2A60E083E090E00E944C2A1092360270
:1025F00010923702109238021092390260E084E0A3
:1026000090E00E944C2A60E082E290E00E944C2A16
:1026100060E085E090E00E944C2A60E086E090E077
:102620000E944C2A6FEF87E090E00E944C2A40E025
:1026300050E0BA0188E090E00E945E2A60E08DE000
:1026400090E00E944C2A40E050E0BA0188E190E01E
:102650000E945E2A60E087E190E00E944C2A40E000
:1026600050E0BA018CE190E00E945E2A60E070E0E8
:1026700080E290E00E946A2A40E050E0BA0188E1DE
:1026800090E00E945E2A0C94DF120C94E612682FF0
:102690008EE090E00C944C2A0E941C2260939402DD
:1026A00070939502809396029093970260939002A4
:1026B000709391028093920290939302089585B74C
:1026C000806885BF85B7806885BF089581E00895DB
:1026D0000C94661308950C946A130C946A130C946A
:1026E0006D130C946A130C9471130C946A130E946A
:1026F0005F1381E494E20E948E200E9475130C9473
:1027000073130E946B130C946A130E9434160C947A
:10271000E6070E9407220E945F170E9485130C940F
:102720006F135F926F927F928F929F92AF92BF9240
:10273000CF92DF92EF92FF920F931F93CF93DF938D
:10274000CDB7DEB72A970FB6F894DEBF0FBECDBF68
:102750000E947417C82E81110E944C1336E8832EF4
:1027600032E0932E00E010E0502E802F0E94581689
:102770005C01F401619071904F0168267926611423
:102780007104B1F40F5F1F4F0530110569F78FEF2A
:1027900089838A831B820E9410228160782F9D8307
:1027A0008C8349815A816B818D810E9429083AC0AE
:1027B0008091980281FD0E946116D12CEE24E39451
:1027C000F12CC3018E219F21892B29F10E946813CE
:1027D0008823A9F0DE825F82AE20BF2081E0AB2893
:1027E00009F480E088870E9410228160782F9A8700
:1027F00089874E815F8168858A850E942908000F3C
:10280000111FF801EA57FD4F80819181E826F926D2
:10281000F182E08207C0D394EE0CFF1CFFE0DF12D0
:10282000D0CFB0CF81E0C11001C080E02A960FB6B2
:10283000F894DEBF0FBECDBFDF91CF911F910F91F6
:10284000FF90EF90DF90CF90BF90AF909F908F90D0
:102850007F906F905F9008950E9491130E94FD19E0
:102860000C94F707CF93DF930E945C15EC01811560
:1028700021E5920708F045C0811530E5930708F07F
:1028800094C0883E910528F5803E910508F0F8C077
:10289000883A910570F4853A910508F07CC0813042
:1028A000910509F475C008F4E8C0049708F0E8C081
:1028B000E4C08F3B910508F0E0C0C85AD0E0CC0FCF
:1028C000DD1FC65BDE4F0990D881C02DCE01946418
:1028D000D8C0811540E2940758F4811551E095075E
:1028E00008F0CEC08D3E910508F4C7C09065C9C000
:1028F000C11580E4D80708F4C0C0DF70CE01906A2B
:10290000C0C0811525E59207A8F4811534E5930729
:1029100008F095C0811543E5940708F07BC0811548
:1029200052E5950708F061C0D82FCC27CE01816F02
:10293000906AA7C0C11589E5D807A0F4C11528E59C
:10294000D20708F082C0C11536E5D30708F095C05C
:102950008C2F0E94F0158F7190E0D82FCC27CE01DC
:1029600090628FC0C1154AE5D40708F474C0CE0147
:1029700090568115904208F080C08D2F8F710E9473
:10298000F015DD27D0628F71AE01582BCA0179C0D6
:1029900081E090E076C0C55AD0E0C858DE4F88810B
:1029A000C82FD0E0CE0190646CC074E096958795F6
:1029B0007A95E1F7282F23703C2F337081E090E067
:1029C00002C0880F991F3A95E2F79C68AC01522B20
:1029D0009A019C2F9F709695969550E2959FE001E5
:1029E0001124C9018C2B9D2B4CC08370992721E0A9
:1029F00030E002C0220F331F8A95E2F79C2F969594
:102A0000969580E2989FE0011124C22BD32BCE0132
:102A10009C6837C08370992721E030E002C0220F04
:102A2000331F8A95E2F79C2F9695969540E2949FE6
:102A3000E0011124C22BD32BCE019A6822C0D82FDB
:102A4000CC27CE01846F906A1CC0DC2FCC27CE012E
:102A5000806F906A16C08C2F8F700E94F01594E0E2
:102A6000D695C7959A95E1F7CF70D0E0DC2FCC27AB
:102A7000D0699E01282BC90104C080E090E001C00C
:102A8000CE01DF91CF9108952BE4829FC0011124E4
:102A9000FC012FE0729FE00DF11D1124E60FF11DE6
:102AA000EE0FFF1FE852FF4F8591949108950E9409
:102AB00044150E94321408958238910569F1B0F4EA
:102AC0008133910509F46DC048F48932910509F408
:102AD00063C08A32910509F469C008958533910570
:102AE00009F455C089339105B9F00895833E9105E5
:102AF00069F138F4803E9105B1F0823E910509F10B
:102B00000895863E9105A9F1873E9105B9F1843E6D
:102B1000910509F064C023C02091CB0220FD4FC075
:102B200021FD4DC008958091CB0280FD44C080916D
:102B3000CC0280FF44C08091CB0284FD42C083EE72
:102B40004DC08091CB0282FF38C0F5CF8091CB027F
:102B500082FD33C08091CC0280FD31C0ECCF8091EA
:102B6000CC0281FF32C08091CB0284FD2AC087EE67
:102B700035C08091CB0283FF26C0F5CF8091CB0278
:102B800083FD21C08091CC0281FD1FC0ECCF8091DC
:102B9000CB0285FD1CC01DC08091CB0285FD19C0F4
:102BA00016C08091CB0286FD16C017C08091CB0263
:102BB00086FD13C010C089E311C082EE0FC080EE05
:102BC0000DC080E00BC086EE09C084EE07C089E22C
:102BD00005C085E303C08AE201C081E390E0089567
:102BE0009091CB0292FF0DC0282F2871283019F444
:102BF000877F846006C0282F2471243011F48B7FD6
:102C0000886093FF0DC0282F2871283119F4877E22
:102C1000846106C0282F2471243111F48B7E8861D1
:102C20002091CC0220FF0DC0382F3871383019F4B4
:102C3000877F816006C0382F3171313011F48E7F6B
:102C4000886021FF0DC0282F2871283119F4877E54
:102C5000816106C0282F2171213111F48E7E886197
:102C600094FD877E089508950E949D12811102C0EF
:102C70000E9445130E94A812809398020E94B012ED
:102C80009093CC028093CB020E9433160E94AC1228
:102C9000682F70E080E090E00E94AB0C60913202FF
:102CA0007091330280913402909135020C94E30CC0
:102CB000E82FF0E0EE0FFF1FE952FD4F8081918178
:102CC0000895CF92DF92EF92FF920F931F93CF93CD
:102CD000DF938AE893E00E94390687EDE82E82E0D0
:102CE000F82EC0E0D0E095E8C92E93E0D92E0CE78D
:102CF00013E0DF93CF93DF92CF920E94D20682E857
:102D000093E00E943906F701819191917F010E9421
:102D1000CC079F938F931F930F930E94D2068AE74D
:102D200093E00E94390621968DB79EB708960FB69C
:102D3000F8949EBF0FBE8DBFC530D105D1F6DF918F
:102D4000CF911F910F91FF90EF90DF90CF9008955A
:102D500080EA8A95F1F7089500C008950C94A816AA
:102D600008950C94B0160C94B1160C94B0160C94F3
:102D7000B516F894E82FE295EF70F0E031A1282F16
:102D80002F7081E090E001C0880F2A95EAF7982F14
:102D90009095932391A392A1892B82A3789408956F
:102DA0000F931F93CF93DF93CAE8D1E089918F3FB0
:102DB00011F00E94B91681E0CF38D807B9F7CBE7F8
:102DC000D1E00AE811E089918F3F11F00E94B91615
:102DD0000C171D07C1F7DF91CF911F910F91089537
:102DE000BF92CF92DF92EF92FF920F931F93CF93F8
:102DF000DF938C01C62FD0E0CE0186579E4F6C0129
:102E0000FC0190819F3F09F450C0B62EF894E92F41
:102E1000E295EF70F0E081A19F7021E030E001C009
:102E2000220F9A95EAF7822B81A382A1209528236D
:102E300022A378940E94AC16EBE7F1E04AE851E057
:102E400021E030E0E12CF12C61916F3F89F0A62F59
:102E5000A295AF70B0E090968C9190E06F7002C038
:102E6000959587956A95E2F780FD02C0C90102C079
:102E700080E090E0E82AF92A220F331F4E175F07FF
:102E800019F7F60180818F3F11F00E94B91661E0B9
:102E9000E114F10409F460E08B2D0E94AE16CC0F12
:102EA000DD1FC00FD11FF982E882DF91CF911F9102
:102EB0000F91FF90EF90DF90CF90BF9008950E9408
:102EC000D0168AE0E7EDF2E0DF01982F1D929A9587
:102ED000E9F7EDECF2E0DF011D928A95E9F785E074
:102EE0000E94BF170C942D07FF920F931F93CF934F
:102EF000DF93CDB7DEB72A970FB6F894DEBF0FBECB
:102F0000CDBF8E010F5F1F4F8AE0F80111928A95A5
:102F1000E9F7F12C6F2DC8010E94F016F394F5E04B
:102F2000FF12F8CF4AE050E0B8018DEC92E00E9429
:102F3000312AFF24F394009709F4F12C892B41F0F6
:102F40008AE0F801ADECB2E001900D928A95E1F7CC
:102F50002F2D45E067ED72E08DEC92E00E94C017E6
:102F60000E942F078F2D2A960FB6F894DEBF0FBE52
:102F7000CDBFDF91CF911F910F91FF9008950895DC
:102F8000FF920F931F93CF93DF93F82E092F162FE5
:102F9000D72FC42F222349F081E080939B020E9407
:102FA000102290939A028093990280919B02882329
:102FB000D9F08091990290919A020E942822059757
:102FC00098F0EF2DF02FA12FBD2F80E090E04C2F37
:102FD00050E08417950734F4219131912D933D935E
:102FE0000196F7CF10929B02DF91CF911F910F9125
:102FF000FF9008950E94BD240E9489130C94C92457
:103000000E94CD240E942C140C94EB240E94AE212B
:103010000E94A4240E9477130E94FA170E940018AD
:103020000E948113FBCF8091A20280FF06C06091B5
:10303000090170E0660F771F26C081FF04C0609110
:10304000090184E005C082FF07C06091090188E0A2
:10305000689FB001112417C09091A1029923D1F06B
:1030600060910801961788F72091090188E0289F50
:1030700090011124929FA001939F500D112470E0A4
:10308000CA010E94032A6038710540F46115710578
:1030900019F406C068E070E0862F08958FE7089560
:1030A00081E008958091A20280FF08C0609105012F
:1030B00070E0759567957595679521C081FF06C08D
:1030C0006091050170E07595679519C082FF04C095
:1030D0006091050170E010C09091A002992399F0D1
:1030E000609104019617A0F780910501899FC001A6
:1030F000112470E00E94032A6038710540F46115C4
:10310000710519F406C061E070E0862F08958FE71D
:10311000089581E008958D3E21F40E941318819551
:1031200004C08E3E29F40E9413188093A6020895CD
:103130008F3E21F40E941318819504C0803F29F42A
:103140000E9413188093A5020895893F19F40E94E4
:10315000521805C08A3F31F40E945218819580931D
:10316000A70208958B3F21F40E945218819504C054
:103170008C3F29F40E9452188093A80208959FE082
:10318000980F983078F421E030E0A90102C0440F94
:10319000551F9A95E2F7CA019091A402892B80935A
:1031A000A40208958D3F21F48091A20281600BC09A
:1031B0008E3F21F48091A202826005C08F3F29F4E6
:1031C0008091A20284608093A20208958D3E39F41A
:1031D0009091A60297FF35C01092A60259C08E3E6C
:1031E00029F49091A6021916BCF32BC09091A50268
:1031F0008F3E29F497FF25C01092A50249C0803F59
:1032000019F41916CCF31DC09091A702893F29F437
:103210001916BCF41092A7023BC08A3F19F497FF1D
:1032200010C0F8CF8B3F39F49091A80297FF09C0E6
:103230001092A8022DC08C3F21F49091A80219167B
:10324000BCF39FE0980F983080F421E030E0A901B2
:1032500002C0440F551F9A95E2F7CA0180959091DC
:10326000A40289238093A40213C08D3F21F480918E
:10327000A2028E7F0BC08E3F21F48091A2028D7F2F
:1032800005C08F3F29F48091A2028B7F8093A20218
:103290008091A502811106C08091A602811102C011
:1032A0001092A1028091A702811106C08091A8020C
:1032B000811102C01092A00208958091980283FFAC
:1032C0007EC088EC93E00E9439068091A4021F9290
:1032D0008F9383EC93E09F938F930E94D20681ECAF
:1032E00093E00E9439068091A502282F082E000C39
:1032F000330B3F938F938EEB93E09F938F930E94BA
:10330000D2068CEB93E00E9439068091A602282F0A
:10331000082E000C330B3F938F9389EB93E09F9320
:103320008F930E94D20687EB93E00E94390680912A
:10333000A702282F082E000C330B3F938F9384EBAA
:1033400093E09F938F930E94D20682EB93E00E94BA
:1033500039068091A802282F082E000C330B3F93CA
:103360008F938FEA93E09F938F930E94D2068CEA0B
:1033700093E00E9439068091A1021F928F9389EAFF
:1033800093E09F938F930E94D20687EA93E00E9476
:1033900039068091A2021F928F9384EA93E09F9353
:1033A0008F930E94D20681EA93E00E9439068DB77E
:1033B0009EB74C960FB6F8949EBF0FBE8DBF0E946D
:1033C00010222091A502211104C02091A6022223DF
:1033D00021F090939F0280939E022091A7022111D9
:1033E00004C02091A802222321F090939D02809393
:1033F0009C0283EA92E00C94ED20EF92FF920F93EF
:103400001F93CF93DF9300D000D000D0CDB7DEB7AD
:1034100086E0E3EAF2E0DE01119601900D928A95D2
:10342000E1F7E090A502F090A6020091A7021091AA
:10343000A8021092A5021092A6021092A702109262
:10344000A802E11003C0FF2009F45DC080919E0234
:1034500090919F020E942822AC019091A102992391
:1034600039F020910A0130E02417350758F04BC09D
:1034700020910B018AE0289F900111242417350721
:1034800018F041C09F3F19F09F5F9093A102EE207A
:1034900061F00E9413181E1414F09FEF01C091E018
:1034A000989F902D11249093A502FF2061F00E9417
:1034B00013181F1414F09FEF01C091E0989F902DF6
:1034C00011249093A6023091A5023323E1F02091BC
:1034D000A6022223C1F045EB3403C0011124992335
:1034E00019F09093A50203C081E08093A50235EB0B
:1034F0002303C0011124992319F09093A60203C05D
:1035000081E08093A602011103C0112309F45DC07C
:1035100080919C0290919D020E942822AC01909182
:10352000A002992339F02091060130E024173507D5
:1035300058F04BC0209107018AE0289F9001112488
:103540002417350718F041C09F3F19F09F5F9093F3
:10355000A002002361F00E945218101614F09FEF91
:1035600001C091E0989F902D11249093A702112300
:1035700061F00E945218111614F09FEF01C091E003
:10358000989F902D11249093A8023091A702332385
:10359000E1F02091A8022223C1F045EB3403C001E1
:1035A0001124992319F09093A70203C081E080931E
:1035B000A70235EB2303C0011124992319F090933E
:1035C000A80203C081E08093A8028091A502811126
:1035D0000BC08091A602811107C08091A7028111C2
:1035E00003C08091A80281110E945D19EB82FC82C8
:1035F0000D831E8386E0FE013196A3EAB2E00190BE
:103600000D928A95E1F726960FB6F894DEBF0FBEAD
:10361000CDBFDF91CF911F910F91FF90EF90089553
:10362000E3EAF2E086E0DF011D928A95E9F7109265
:10363000A1021092A0021092A2020895CF93DF93EC
:10364000EC01FB018281882309F43CC1C430FDE513
:10365000DF0760F4CB3F9CE5D90788F49E01225038
:103660003C452431310508F02EC109C0C236EDE5D4
:10367000DE0729F0C63AFDE5DF0709F024C10E9404
:10368000B0129093CC028093CB02C1318CE5D80765
:1036900009F4C6C008F042C0C930ECE5DE0709F401
:1036A0009BC000F5C5308CE5D80709F485C078F4D7
:1036B000C330ECE5DE0709F478C008F07AC0C23008
:1036C000DC4509F0F5C08091CB028160EFC0C730C6
:1036D0009CE5D90709F478C008F07AC08091CB0244
:1036E0008061E4C0CD30FCE5DF0709F487C058F401
:1036F000CB309CE5D90709F479C008F07BC08091F4
:10370000CB0288606FC0CF30FCE5DF0709F480C0D2
:1037100008F082C08091CB02877FC8C0CE3F9CE575
:10372000D90709F471C000F5C531FCE5DF0709F4DC
:1037300085C068F4C3319CE5D90709F475C008F069
:1037400095C00E94530C8091CB028F77AFC0CC3FC5
:10375000FCE5DF07A9F108F054C0CB3FDC4509F0D8
:10376000A7C08091CC0240C0C230EDE5DE0709F46D
:1037700089C058F4C1158DE5D80709F45AC008F07E
:1037800069C08091CC0282602FC0C236EDE5DE07B1
:1037900009F47CC0C63AFDE5DF0709F481C0C330F7
:1037A000DD4509F085C080E06EC08091CB0282606B
:1037B0007DC08091CB0216C08091CB02886076C01C
:1037C0008091CC0282604FC08091CB0280626EC03B
:1037D0008091CB0280646AC00E94530C8091CB021E
:1037E000806864C0846062C081603DC08091CB020B
:1037F0008E7F5CC08091CB028D7F58C08091CB02C0
:1038000016C08091CC0218C08091CC028D7F2BC055
:103810008091CB028F7E4AC08091CB028F7D46C0C3
:103820008091CB028F7B42C08091CB02877F8B7FC0
:103830003DC08091CC028D7F8E7F15C08091CB02E0
:1038400082FB222720F991E0922790FB82F990FBDE
:1038500083F92CC08091CC02982F909591708E7F27
:10386000892B90FB81F98093CC0222C00E94530CDB
:103870008091CB0287FB222720F991E0922790FBD1
:1038800087F914C081E00E94471312C08091CB02D7
:1038900084FB222720F991E0922790FB84F906C04F
:1038A0008091CB02982F909590FB80F98093CB026A
:1038B0008091CB029091CC020E94C1120E94530CC5
:1038C00080E001C081E0DF91CF91089580910401F3
:1038D0001F928F93809105011F928F938091080111
:1038E0001F928F93809109011F928F9380910A01FB
:1038F0001F928F9380910B011F928F938BEE93E019
:103900009F938F930E94D2068DB79EB70E960FB6E7
:10391000F8949EBF0FBE8DBF0895883220F58E317A
:1039200008F068C08B3091F1C0F4873009F0BEC058
:1039300081E080930B0184E180930A018AE0809307
:1039400009018EE18093080188E08093050188E2F7
:10395000809304018DE495E0C6C0833109F443C02F
:10396000843169F1A3C08F3409F49EC028F48932F0
:1039700031F1883359F09AC0813531F008F4D4C060
:10398000823509F4A7C092C08FEFA5C08FE695E0FD
:103990000E9439060E94661C1F9281E08F931F923D
:1039A00088E08F9388E694E09F938F930E94D206DD
:1039B0000F900F900F900F900F900F9096C08CE685
:1039C00095E00E9439068091AD02882309F4AAC0CF
:1039D0001092AD021092AC021092AB021092AA02A9
:1039E0001092A902B1C08EE595E00E9439060E94AE
:1039F000661C7BC08D518093AD02833031F170F431
:103A00008130D1F0823009F03FC08AE091E090939C
:103A1000AC028093AB028CE991E01FC0853059F174
:103A200008F1863089F584E091E09093AC028093B0
:103A3000AB0287ED91E011C08BE091E09093AC0276
:103A40008093AB0283E991E008C089E091E0909314
:103A5000AC028093AB0288EA91E09093AA02809333
:103A6000A90218C088E091E09093AC028093AB0269
:103A700085EB91E0F2CF85E091E09093AC028093EA
:103A8000AB0284EC91E0E9CF1092AD028BE595E0BA
:103A90000E9439068091AD02882309F455C01F9217
:103AA0008F9387E595E00DC08AE015C08AE495E024
:103AB0001AC097FF47C0108280811F928F9384E4C1
:103AC00095E09F938F930E94D2060F900F900F90D6
:103AD0000F900BC081E0E091AB02F091AC02309707
:103AE00029F581E495E00E9439062091AD02222358
:103AF00059F18091A9029091AA02009711F48FE8E0
:103B000091E09F938F931F922F9388E395E09F936B
:103B10008F930E94D2060F900F900F900F900F90EE
:103B20000F9016C080E0089586EFD5CF2081082E33
:103B3000000C990B820F911D8F3F910509F00CF439
:103B4000B8CF8FEF8083B8CF84E395E00E94390629
:103B500081E00895CF93C82F1F928F9385E895E059
:103B60009F938F930E94D20681E090E0A0E0B0E0A6
:103B7000BC01CD0104C0660F771F881F991FCA952D
:103B8000D2F70E94AB0C0F900F900F900F90CF9137
:103B90000C94530CEF92FF920F931F93CF93DF93EC
:103BA0008B3109F4EDC008F08EC08B3009F4B1C040
:103BB00008F078C0863009F4AFC020F4853009F4ED
:103BC000BDC04EC1873009F4C0C0883009F048C17B
:103BD0000E94AC121F928F938EEA99E09F938F936D
:103BE0000E94D2060E94A81283FB992790F91F9287
:103BF0009F9382FB992790F91F929F9381FB9927AE
:103C000090F91F929F93982F91701F929F931F92EC
:103C10008F9385E699E09F938F930E94D2060E942E
:103C2000B01287FB222720F91F922F9386FB2227B1
:103C300020F91F922F9385FB222720F91F922F93A3
:103C400084FB222720F91F922F9383FB222720F940
:103C50001F922F9382FB222720F91F922F9391FB13
:103C6000222720F91F922F93292F21701F922F9323
:103C700081FB222720F91F922F93282F21701F925A
:103C80002F939F938F9380E898E09F938F930E9448
:103C9000D2068DB79EB788960FB6F8949EBF0FBE1A
:103CA0008DBF35C0803109F495C020F48E3009F401
:103CB0007BC0D6C0863109F4A8C0893109F0D0C0D4
:103CC00085EF95E084C08A32E1F060F4873209F430
:103CD000C3C028F48E3108F4C3C08D51BEC08932F0
:103CE00069F1BEC0833448F48A3308F0B3C0853329
:103CF00009F4B2C0883369F0B3C0833409F4ACC0AE
:103D0000AFC089E59AE00E9439060E944513C1E0E0
:103D1000ACC08DED96E05BC080919802817F8E7F74
:103D20008093980286EB96E00E94390685E59AE03A
:103D30000E94390681E08093AE02E9CF89E39AE0E0
:103D40000E9439060E943207E2CF80919802C82F64
:103D5000C095C170C0FB80F980939802CC2329F0F4
:103D60008DE29AE00E94390680C080E29AE00E94CB
:103D7000390680919802897F877F80939802C7CF08
:103D80009091980291FBCC27C0F981E0C827892F38
:103D9000C0FB81F980939802CC2319F083E19AE06B
:103DA00029C085E09AE013C09091980292FBCC273D
:103DB000C0F981E0C827892FC0FB82F9809398025F
:103DC000CC2319F086EF99E015C086EE99E00E94A9
:103DD00039069DCF9091980293FBCC27C0F981E0E2
:103DE000C827892FC0FB83F980939802CC2351F018
:103DF0008AED99E00E943906809198028160809353
:103E0000980233C08DEC99E0E2CF0E941C22162F5D
:103E1000072FF82EE92ED091CA02C09118010E94F6
:103E20009820EF92FF920F931F931F92DF931F92A0
:103E3000CF931F928F938AE895E09F938F930E9470
:103E4000D2068DB79EB70C960FB6F8949EBF0FBEE4
:103E50008DBF5DCF895301C080E00E94AA1D57CF5E
:103E60008BEC99E00E943906C0E08C2FDF91CF9156
:103E70001F910F91FF90EF90089580E008950C94AA
:103E80003D1FCF93C82F8091AE02813071F040F07A
:103E9000823009F045C08C2F0E948D1C81E046C005
:103EA0000E94A6118232F1F504C00E94A61182324E
:103EB00061F48C2F0E943F1F811104C08C2F0E943F
:103EC000CA1D2CC081E090E029C08C2F0E943D1FAC
:103ED000811123C0C431C9F058F4CB3069F0C0312E
:103EE000B9F482E08093AE0288E30E948D1C15C075
:103EF000C93259F0C83361F486EB96E00E94390666
:103F000081E895E00E94390608C01092AE020CC00C
:103F10008FE795E00E94390607C081E0817006C0F6
:103F20001092AE0280E002C080E0F8CFCF910895F9
:103F3000CF93DF9386319C4541F5EB010E94A6119A
:103F4000982F8A812091020130910301882379F012
:103F50009A7A81E009F480E08093AF02911102C067
:103F600069E201C065E3C9010E9469210AC080912C
:103F7000AF02811102C069E201C065E3C9010E947C
:103F80006B210E94E81180E001C081E0DF91CF91B8
:103F900008950F931F93CF93DF93C42FD22FFC016B
:103FA00082818823C9F04093B2020E94102290932C
:103FB000B1028093B00280E28C0F883008F057C0C5
:103FC000C77081E001C0880FCA95EAF7DF91CF91F1
:103FD0001F910F910C94B0098091B202481330C028
:103FE0008091B0029091B1020E942822883C9105F4
:103FF00038F510E21D0FCD17B9F080E28C0F883034
:1040000040F4C77081E001C0880FCA95EAF70E94AA
:10401000B709183028F581E09D2F977001C0880FEF
:104020009A95EAF70E94B009802F0E94A7091830DC
:10403000F0F4D77081E001C0880FDA95EAF70AC082
:1040400080E28C0F883098F4C77081E001C0880F3F
:10405000CA95EAF7DF91CF911F910F910C94B709A0
:10406000802FDF91CF911F910F910C94A709DF91C1
:10407000CF911F910F9108950F939C01CB01243F85
:104080004CE5340731F188F4293DFCE53F07D9F0D0
:104090002A3D4CE5340779F1283D3C45A9F506E277
:1040A00021EE41EE68ED7CE52BC0263FFCE53F07A5
:1040B000E1F0A8F0273F3C4539F507E225EE46EE52
:1040C00067EF7CE51DC007E225EE45EE69ED7CE576
:1040D00017C006E221EE40EE64EF7CE511C007E276
:1040E00025EE44EE65EF7CE50BC006E221EE42EEE4
:1040F00066EF7CE505C008E221E045EE6AED7CE56F
:104100000E94C91F80E008C0FC018281882319F049
:104110001092B20201C081E00F9108959093FD01C9
:104120008093FC0108959093B8028093B70208959C
:10413000E091B702F091B802309721F00190F08140
:10414000E02D099480E00895EF92FF920F931F9362
:10415000CF93DF93E091B702F091B8023097B1F1BD
:104160008C010280F381E02D09958091980282FFF5
:104170002DC080FF04C082E79AE00E943906E80162
:1041800018E08CE6E82E8AE0F82E8091980280FFF5
:104190000BC088811F928F93FF92EF920E94D206EC
:1041A0000F900F900F900F90115021961111EDCF9D
:1041B0008091980280FF0AC08AE69AE0DF91CF9151
:1041C0001F910F91FF90EF900C943906DF91CF91E2
:1041D0001F910F91FF90EF900895E091B702F09139
:1041E000B802309739F022E0DC012C930480F5818D
:1041F000E02D099408952091B5023091B602281758
:10420000390771F09093B6028093B502E091B7023E
:10421000F091B802309721F00680F781E02D0994E3
:1042200008952091B3023091B4022817390771F034
:104230009093B4028093B302E091B702F091B80278
:10424000309721F00084F185E02D09940895FC0158
:10425000329697E080E0915029F021912223D9F302
:104260008F5FF9CF0895662349F0FC0132960896D6
:104270002191621729F0E817F907D1F780E0089536
:1042800081E008959C01FC0132969FEF80E041910E
:10429000461789F09F3F19F4411101C0982F8F5F95
:1042A0008630A9F79F3F39F0F901E90FF11D97FD1D
:1042B000FA956283089508959C012A5F3F4FFC019F
:1042C0004281461301C01282019682179307B9F703
:1042D00008950C9442210C945C21029626E0FC0186
:1042E00011922A95E9F7089508950C94742183E0BA
:1042F0008093B9020C947521811102C081E001C044
:1043000082E08093B9020C9475210C947C2181E0A9
:104310008093B9020C9475210C94872108950C9414
:104320008E210C948F210C948E210C948E210C9450
:104330008E21CF930E9495210E9474170E94932191
:10434000C0E08C2F0E945816892B29F4CF5FC5300E
:10435000C1F780E001C081E0CF91089508951F92D8
:104360000F920FB60F9211248F939F93AF93BF9329
:104370008091BA02811113C08091E1029091E20212
:10438000A091E302B091E4024196A11DB11D80937A
:10439000E1029093E202A093E302B093E402BF91A2
:1043A000AF919F918F910F900FBE0F901F90189516
:1043B0008091E902843031F10E94B2071092BA0272
:1043C00020E488E190E00FB6F894A895809360000F
:1043D0000FBE2093600083B7817F846083BF83B763
:1043E000816083BF7894889583B78E7F83BF0FB633
:1043F000F894A89580916000886180936000109285
:1044000060000FBE08950E94530C0C94B60782E022
:1044100084BD93E095BD9AEF97BD80936E0008959B
:104420002FB7F8948091E1029091E202A091E3020B
:10443000B091E4022FBF08952FB7F8946091E10284
:104440007091E2028091E3029091E4022FBF0895FF
:104450009C014FB7F8948091E1029091E202A09103
:10446000E302B091E4024FBF821B930B089578944E
:104470001F920F920FB60F9211248F939F93AF93B9
:10448000BF938091E1029091E202A091E302B0918A
:10449000E4020196A11DB11D8093E1029093E20216
:1044A000A093E302B093E402BF91AF919F918F91EB
:1044B0000F900FBE0F901F90189587E797E7909386
:1044C0000108809300089AE088E10FB6F894A89557
:1044D000809360000FBE90936000FFCF8091C9026F
:1044E0000895089522E02093E9002FEF3091E8002D
:1044F000215035FD06C035ED3A95F1F70000211148
:10450000F5CF2091E80025FF0BC040E050E066E0C9
:1045100070E00E945A258091E8008E778093E80031
:104520000895CF93DF9321E02093E9002FEF30919E
:10453000E800215035FD06C035ED3A95F1F7000051
:104540002111F5CF2091E80025FF14C0EC0140E0D7
:1045500050E068E070E00E945A258091E8008E7774
:104560008093E80088E0FE01A1ECB2E001900D929A
:104570008A95E1F7DF91CF9108958093BD02709302
:10458000BF026093BE028091E902843001F582E0AF
:104590008093E9008FEF9091E800815095FD06C06F
:1045A00095ED9A95F1F700008111F5CF8091E80023
:1045B00085FF0DC040E050E063E070E08DEB92E0DD
:1045C0000E945A258091E8008E778093E800089534
:1045D000BC0184E00C94BD22BC0183E00C94BD229C
:1045E00088E99AE00E9439068091E802811109C0A9
:1045F0000E94EB260E9448278091E200846080930D
:10460000E200089584E99AE00E9439061092E802D7
:10461000089580E99AE00E9439060C948C218CE878
:104620009AE00E9439066091E50281E0611101C0C3
:1046300080E00C94772188E89AE00E9439069091F6
:10464000E90281E0943009F080E06091E5020C9489
:104650007C212091BC022F5F822F62E30E94F72908
:10466000992319F02093BC0208951092BC02809106
:10467000C002882371F18091E902843041F5809174
:10468000E9008F702091EC00922F917020FD90E84E
:10469000892B93E09093E9009091EB0090FF14C078
:1046A0009091EE0097FF10C09091E80095FF03C035
:1046B0001092F100F9CF9091E80090FF05C0909121
:1046C000E8009E779093E8008F708093E900109245
:1046D000C002089542E061EC81E00E94642642E25B
:1046E00061EC82E00E94642642E261EC83E00E9479
:1046F00064269091E90281E0943009F080E06091B5
:10470000E5020C9485218091EB02833009F461C0AD
:1047100030F4813071F0823009F49AC008958A3003
:1047200009F486C08B3009F46CC0893009F0A8C048
:1047300020C08091EA02813A09F0A2C08091E8008D
:10474000877F8093E8008091EE029091EF02892BA1
:1047500021F468E081EC92E003C060E080E090E04A
:1047600070E00E94A5258091E8008B778093E80097
:1047700008958091EA02813209F082C08091EE02B0
:104780009091EF02029708F07BC08091E800877F4C
:104790008093E8008091E80082FD05C08091E902E5
:1047A0008111F8CF6DC02091F3008091F20090E06C
:1047B000922B029731F48091F100813011F0863014
:1047C00021F48091F1008093C9028091E8008B77F9
:1047D00053C08091EA02813A09F052C08091EE0202
:1047E0009091EF02892B09F04BC08091E800877F00
:1047F0008093E8008091E80080FFFCCF8091180151
:1048000036C08091EA028132D9F58091EE02909112
:10481000EF02892BA9F58091E800877F8093E8005B
:104820000E9499268091EC02809318010C94530CFD
:104830008091EA02813221F58091E800877F8093A0
:10484000E8000E9499268091ED028093CA020895A3
:104850008091EA02813AA1F48091E800877F8093F9
:10486000E8008091E80080FFFCCF8091CA0280932D
:10487000F1008091E8008E778093E8000C949926EF
:1048800008959FB7F8941092C0029FBF9091E902DB
:10489000943009F057C09091E9009F703091EC007E
:1048A000232F217030FD20E8922B23E02093E90094
:1048B0002091EB0020FF43C02091EE0027FF3FC076
:1048C0002091BB02222321F02091E80025FF37C070
:1048D0001092BB0226E03091E80035FD15C0309102
:1048E000E902343061F53091EB0035FD28C02150EC
:1048F00021F481E08093BB0222C0EFE9FFE0319711
:10490000F1F700C00000E7CF8093F1008091E8004C
:1049100085FD0AC08091E80080FFFCCF8091E8000F
:104920008E778093E80006C08FB7F89421E020933B
:10493000C0028FBF9F709093E90080E008959F7040
:104940009093E9008FEF089584B7877F84BF0FB6F7
:10495000F894A8958091600088618093600010921F
:1049600060000FBE90E080E80FB6F894809361007D
:10497000909361000FBE0C9487210E94EB260E9449
:104980004827E2EEF0E080818460808378940C9484
:10499000DC298CE091E00C9493208091E902853031
:1049A000C9F484E89AE00E9439068091E9028530D2
:1049B00079F40E94D8218091E7028823B1F30E9404
:1049C0009921882391F30E9444250E94530CEDCF36
:1049D0000C940322089508950C94EE24292F332774
:1049E00023303105C9F060F42130310581F02230E7
:1049F000310509F041C08BE590E022ED3AE040C07E
:104A000021323105E1F02232310531F135C082E148
:104A100090E02DE23BE034C099278130910549F0C8
:104A200028F0029749F5ECE9FAE005C0EEECFAE06F
:104A300002C0E0ECFAE0849190E09F0121C0633075
:104A40007105D0F4660F771FFB01EB50FE4F2081FC
:104A5000318189E090E014C06330710568F4FB0196
:104A6000EE0FFF1FE151FE4F20813181FB01E45128
:104A7000FE4F808190E004C080E090E020E030E0D4
:104A8000FA0131832083089580E189BD82E189BDE7
:104A900009B400FEFDCF8091D8008F7D8093D800AF
:104AA0008091E00082608093E0008091E00081FDD1
:104AB000FCCF0895CF92DF92EF92FF920F931F9356
:104AC000CF93DF93EC018B017A010E94B82681110C
:104AD00033C0E114F10439F0F70180819181081BA2
:104AE000190BC80FD91FC12CD12C0115110519F1B3
:104AF0008091E80085FD16C08091E8008E77809354
:104B0000E800E114F10449F0F70180819181C80EB9
:104B1000D91ED182C08285E00FC00E94B8268823AA
:104B200021F30AC089918093F10001501109FFEF30
:104B3000CF1ADF0ADACF80E0DF91CF911F910F917A
:104B4000FF90EF90DF90CF9008952091F002309188
:104B5000F1022617370748F06115710539F42091E5
:104B6000E8002E772093E80001C0B901FC0120E0A5
:104B70006115710579F18091E9028823F1F18530A1
:104B8000F1F18091E80083FD3CC08091E80082FD56
:104B90002EC08091E80080FFEBCF2091F300809140
:104BA000F20090E0922B6115710551F0883091056B
:104BB00038F421912093F100615071090196F3CFEF
:104BC00021E0089709F020E08091E8008E7780933B
:104BD000E800CECF2111CFCF0AC08091E90288230F
:104BE00061F0853061F08091E80083FD0AC080911A
:104BF000E80082FFF2CF80E0089582E0089583E02C
:104C0000089581E008952091F0023091F102261775
:104C1000370748F06115710539F42091E8002E77C7
:104C20002093E80001C0B901FC0120E06115710585
:104C300091F18091E902882309F440C0853009F49C
:104C40003FC08091E80083FD3DC08091E80082FD77
:104C50002FC08091E80080FFE9CF2091F300809180
:104C6000F20090E0922B6115710559F088309105A2
:104C700040F424912093F10031966150710901961E
:104C8000F2CF21E0089709F020E08091E8008E77CC
:104C90008093E800CBCF2111CCCF0AC08091E902EC
:104CA000882361F0853061F08091E80083FD0AC0BF
:104CB0008091E80082FFF2CF80E0089582E00895BD
:104CC00083E0089581E00895982F973068F59093D8
:104CD000E900981739F07091EC002091ED005091A7
:104CE000F00003C0242F762F50E021FD02C09F5F0B
:104CF000ECCF3091EB003E7F3093EB003091ED0034
:104D00003D7F3093ED003091EB0031603093EB004C
:104D10007093EC002093ED005093F0002091EE0092
:104D200027FDE5CF80E008958F708093E90081E052
:104D300008958091EA0287FF11C08091E80082FD0A
:104D400005C08091E9028111F8CF11C08091E8007F
:104D50008B770BC08091E902882349F08091E800AD
:104D600080FFF8CF8091E8008E778093E800089567
:104D70002091E4003091E50095E64091EC00842F0D
:104D8000817040FF23C08091E80080FD1DC08091AC
:104D9000E902882399F0853099F08091EB0085FD38
:104DA00011C04091E4005091E5002417350729F324
:104DB000915011F09A01E1CF84E0089582E00895C6
:104DC00083E0089581E0089580E008954091E8002F
:104DD00042FFDDCF08950E9459270E946127E0EE2F
:104DE000F0E0808181608083E8EDF0E080818F7762
:104DF000808319BCA7EDB0E08C918E7F8C9380816D
:104E00008F7E80831092E80208950F931F93CF93B3
:104E1000DF930E9459270E946127C8EDD0E0888166
:104E20008F77888388818068888388818F7D888355
:104E300019BC1092E9021092E5021092E70210925A
:104E4000E60200EE10E0F80180818B7F808388818C
:104E50008160888342E060E080E00E946426E1EEA9
:104E6000F0E080818E7F8083E2EEF0E080818160DF
:104E70008083808188608083F80180818E7F808339
:104E8000888180618883DF91CF911F910F91089570
:104E9000E8EDF0E080818F7E8083E7EDF0E08081B7
:104EA0008160808384E082BF81E08093E8020C947B
:104EB0000527E8EDF0E080818E7F80831092E2008C
:104EC00008951092DA001092E10008951F920F9257
:104ED0000FB60F9211242F933F934F935F936F93CD
:104EE0007F938F939F93AF93BF93EF93FF938091A3
:104EF000E10082FF0BC08091E20082FF07C0809139
:104F0000E1008B7F8093E1000E9429238091DA00E9
:104F100080FF1FC08091D80080FF1BC08091DA0005
:104F20008E7F8093DA008091D90080FF0DC080E1F0
:104F300089BD82E189BD09B400FEFDCF81E0809387
:104F4000E9020E94F02205C019BC1092E9020E94F9
:104F500002238091E10080FF19C08091E20080FF70
:104F600015C08091E2008E7F8093E2008091E20084
:104F700080618093E2008091D80080628093D800A5
:104F800019BC85E08093E9020E940F238091E10023
:104F900084FF30C08091E20084FF2CC080E189BD95
:104FA00082E189BD09B400FEFDCF8091D8008F7DDC
:104FB0008093D8008091E1008F7E8093E100809102
:104FC000E2008F7E8093E2008091E2008160809316
:104FD000E2008091E502882311F084E007C080910F
:104FE000E30087FD02C081E001C083E08093E90215
:104FF0000E941B238091E10083FF29C08091E20081
:1050000083FF25C08091E100877F8093E10082E0EB
:105010008093E9021092E5028091E1008E7F8093F7
:10502000E1008091E2008E7F8093E2008091E200B7
:1050300080618093E20042E060E080E00E946426AC
:105040008091F00088608093F0000E940923FF9116
:10505000EF91BF91AF919F918F917F916F915F91F0
:105060004F913F912F910F900FBE0F901F90189569
:105070001F920F920FB60F9211242F933F934F93CD
:105080005F936F937F938F939F93AF93BF93CF93D0
:10509000DF93EF93FF93C091E900CF708091EC0014
:1050A000D82FD17080FDD0E81092E9008091F000F7
:1050B000877F8093F00078940E947C281092E9000A
:1050C0008091F00088608093F000CD2BCF70C0936A
:1050D000E900FF91EF91DF91CF91BF91AF919F9147
:1050E0008F917F916F915F914F913F912F910F9091
:1050F0000FBE0F901F9018951F93CF93DF93CDB7DE
:10510000DEB7AA970FB6F894DEBF0FBECDBFEAEEAA
:10511000F2E08091F100819322E0E23FF207C9F7CB
:105120000E9483238091E80083FF2EC18091EA02D0
:105130009091EB02492F50E04A30510508F024C10C
:10514000FA01EE59FF4F0C94172A803821F082386B
:1051500009F01AC108C08091E6029091E7029923F4
:1051600089F082600FC08091EE028F70873008F066
:105170000BC18093E9008091EB0085FB882780F9C3
:105180001092E9009091E800977F9093E800809357
:10519000F1001092F100D1C0282F2D7F09F0F4C04A
:1051A000882319F0823061F0EFC08091EC028130E9
:1051B00009F0EAC0933009F080E08093E7022EC046
:1051C0008091EC0281112AC08091EE028F702FEF46
:1051D000280F263008F0D8C08093E9002091EB001A
:1051E00020FF1CC0933021F48091EB00806214C03A
:1051F0009091EB0090619093EB0021E030E0A901E9
:1052000002C0440F551F8A95E2F74093EA001092BE
:10521000EA008091EB0088608093EB001092E90037
:105220008091E800877F8093E8000E949926ACC0B7
:105230008111AAC01091EC021F778091E300807861
:10524000812B8093E3008091E800877F8093E800C2
:105250000E9499268091E80080FFFCCF8091E300B6
:1052600080688093E300111102C082E001C083E0F6
:105270008093E90289C08058823008F085C080910F
:10528000EC029091ED028C3D53E0950779F583E0B7
:105290008A838AE289834FB7F894DE01139620E06F
:1052A0003EE051E2E32FF0E050935700E49120FFFD
:1052B00003C0E295EF703F5FEF708E2F90E0EA3011
:1052C00010F0C79601C0C0968D939D932F5F243137
:1052D00049F74FBF8091E800877F8093E8006AE23A
:1052E00070E0CE0101960E94A52516C06091EE02E5
:1052F0007091EF02AE014F5F5F4F0E94EC24BC0142
:10530000892B09F441C09091E800977F9093E800C1
:1053100089819A810E9403268091E8008B7780938F
:10532000E80032C0803881F58091E800877F809363
:10533000E8008091E5028093F1008091E8008E778B
:1053400072CF811121C08091EC029091ED029927DA
:105350000297D4F48091E800877F8093E8008091E1
:10536000EC028093E5020E9499268091E50281116A
:1053700006C08091E30087FD02C081E001C084E0A7
:105380008093E9020E946A238091E80083FF0AC0AB
:105390008091E800877F8093E8008091EB00806235
:1053A0008093EB00AA960FB6F894DEBF0FBECDBF78
:1053B000DF91CF911F910895CF938091E9028823C7
:1053C000A1F0C091E900CF709091EC00892F81701D
:1053D00090FD80E8C82B1092E9008091E80083FDE1
:1053E0000E947C28CF70C093E900CF910895991B4B
:1053F00079E004C0991F961708F0961B881F7A95CC
:10540000C9F78095089597FB072E16F4009407D0EE
:1054100077FD09D00E941D2A07FC05D03EF4909527
:1054200081959F4F0895709561957F4F0895EE0F78
:10543000FF1F0590F491E02D0994AA1BBB1B51E1BD
:1054400007C0AA1FBB1FA617B70710F0A61BB70BF4
:10545000881F991F5A95A9F780959095BC01CD0199
:105460000895FB01DC0104C08D910190801921F4A5
:1054700041505040C8F7881B990B0895F999FECF09
:1054800092BD81BDF89A992780B50895A8E1B0E052
:1054900042E050E00C94722A262FF999FECF92BD7B
:1054A00081BDF89A019700B4021639F01FBA20BDE9
:1054B0000FB6F894FA9AF99A0FBE08950396272F1B
:1054C0000E944D2A0E944C2A252F0E944D2A242FEB
:1054D0000C944D2A0196272F0E944D2A0C944C2A99
:1054E000DC01CB01FC01F999FECF06C0F2BDE1BDA4
:1054F000F89A319600B40D9241505040B8F7089593
:04550000F894FFCF4D
:10550400C8007C02280850011E0A14016E22912250
:105514007222EC22E822712201E200E900EA00B5DD
:1055240000B600B700CD008301CC008A019201943B
:10553400012102230224022502260227022A02B3A1
:1055440000B4006F007000818283E200E900EA0089
:10555400B500B600B700CD008301CC008A019201EA
:1055640094012102230224022502260227022A0290
:10557400B300B4006F00700081828397C63435365F
:105584003796F7F6F5F4F1F0333132919094663FA3
:105594003F3F006D6B5F64656C6179006D6B5F69A3
:1055A4006E74657276616C006D6B5F6D61785F73AC
:1055B40070656564006D6B5F74696D655F746F5FC2
:1055C4006D6178006D6B5F776865656C5F6D6178A0
:1055D4005F7370656564006D6B5F776865656C5FAC
:1055E40074696D655F746F5F6D617800407B22DC68
:0C55F4000B610B3F0BE40AFD0A160B00D4
:00000001FF
